:100000000C94E5000C9445110C941E110C94F710FF
:100010000C94D0100C940D010C940D010C94A910AB
:100020000C940D010C9445120C943D0B0C94AF0BE9
:100030000C940D010C940D010C940D010C940D0108
:100040000C940D010C940D010C940D010C940D01F8
:100050000C940D010C940D010C940D010C945F1087
:100060000C940D010C941A0E0C94F40D0C940D01CB
:100070000C940D010C940D010C940D010C940D01C8
:100080000C940D010C940D010C940D010C940D01B8
:100090000C94CC030C940D010C940D010C940D01E7
:1000A0000C940D010C94D0010C940D01190A1C0A3A
:1000B0000B0A0F0A150A3D0A3D0A3D0A200A240AC6
:1000C000280A2E0A320A3D0A380A000000002500DC
:1000D00028002B002E003100000000002300260025
:1000E00029002C002F000404040404030405020268
:1000F00002020403020202020606060606060404C1
:100100000202020404040802011040804010204052
:1001100080408008020401804020100201108010FD
:10012000204040200000000200090F0000030401ED
:10013000000C0000000000000000000000000000B3
:10014000000000080B000202020100090400000187
:10015000020200000524001001052401010104240D
:10016000020605240600010705810310004009046A
:100170000100020A00000007050202400000070516
:1001800083024000000403090412010002EF02018F
:100190004041233680000101020301417264756908
:1001A0006E6F204C4C430041726475696E6F204C39
:1001B000656F6E6172646F0000000000240027000C
:1001C0002A002D0030001421A82011241FBECFEFDB
:1001D000DAE0DEBFCDBF11E0A0E0B1E0E4EDFDE488
:1001E00002C005900D92A63DB107D9F724E0A6ED17
:1001F000B1E001C01D92A235B207E1F710E0C4EEF4
:10020000D0E004C02197FE010E94E823C33ED1073D
:10021000C9F70E9435190C94DD260C94000085ED79
:100220008093BC008091BC0084FDFCCF1092BC0286
:10023000089540912D02262F30E0240F311D2132E8
:100240003105DCF42091BC022430C9F4FC0180E0CB
:1002500090E0861758F430912D022191DC01A55FC2
:10026000BD4FA30FB11D2C930196F3CF80912D02AA
:10027000680F60932D0280E0089581E0089582E088
:1002800008950895E091750280917402E81730F4A2
:10029000F0E0EA58FD4F808190E008958FEF9FEFE6
:1002A00008959091750280917402981750F4E92F87
:1002B000F0E0EA58FD4F208130E09F5F9093750297
:1002C00002C02FEF3FEFC90108958091740290E0C2
:1002D00020917502821B91090895CF92DF92EF92CF
:1002E000FF920F931F93CF93DF937C01262F972FBD
:1002F0008A018091BD02882391F0C62FD72F6E010D
:10030000C40ED51ECC15DD0571F06991D701ED91B4
:10031000FC910190F081E02DC7010995F3CF642F86
:10032000822F0E941901C801DF91CF911F910F9177
:10033000FF90EF90DF90CF900895CF93DF931F92BF
:10034000CDB7DEB769832091BD022223D1F0209181
:10035000DF02203240F021E030E0FC0133832283D1
:1003600080E090E015C08091BE02E82FF0E0E154FB
:10037000FD4F998190838F5F8093BE028093DF024F
:1003800005C061E0CE0101960E94190181E090E074
:100390000F90DF91CF910895089580E090E0089547
:1003A0001F920F920FB60F9211246F927F928F922D
:1003B0009F92AF92BF92CF92DF92EF92FF920F93F4
:1003C0001F932F933F934F935F936F937F938F93DD
:1003D0009F93AF93BF93CF93DF93EF93FF9380915E
:1003E0005A0290915B029C012150310930935B02CB
:1003F00020935A02892B09F0B0C1109272007894B0
:100400008091C100807F84608093C10083E08093ED
:10041000BF0088EE8093D1001092BF001092D200EE
:1004200081E08093190180915C0290915D02892B9B
:1004300009F493C18091540281118FC190900C01F5
:1004400080915302882321F08091520281117BC157
:100450007724739470ECA72E7DE5B72EEAE06E2E1C
:10046000F4E08F2EA0EDCA2EA7E0DA2EB4E0EB2E3A
:10047000F12C04EF11E0CFE0D0E00E949612209121
:100480005C0230915D022F5F3F4F30935D022093FD
:100490005C02853609F45EC07CF5813609F49EC0A5
:1004A00024F58C3309F452C08E3309F44DC08132E7
:1004B00009F08FC080920C01D0920901C09208010E
:1004C000F0920B01E0920A011093070100930601DC
:1004D000D0930501C09304011092530290900C0137
:1004E0008091060190910701C8CF833689F10CF401
:1004F00078C000E022E077C08D36A9F16CF4873631
:1005000079F15CF18C3609F064C00E94B7129093C7
:100510000B0180930A014EC08237D1F14CF48F3623
:1005200009F057C00E94B712982E80930C01A5CFF6
:10053000843789F1863709F04CC00E94B712909336
:1005400005018093040199CF939497CF9A9495CF06
:1005500000E01FC000E024E046C000E025E043C00A
:1005600000E027E040C00E9496128C3619F41092E9
:10057000530204C0709253021092520280915C02A6
:1005800090915D02019690935D0280935C0275CF1D
:1005900001E020E028C00E94B712BC01C5010E9402
:1005A000C023669EC001679E900D1124909309019F
:1005B00080930801809108019091090160910A01DE
:1005C00070910B010E94C023709307016093060194
:1005D00054CF10925D0210925C02BFC000E029E08F
:1005E00002C000E02BE0122F3CE0939E100D11247E
:1005F0000E949612982F977F933259F480915C0253
:1006000090915D02019690935D0280935C021F5F62
:10061000EFCF8D3269F480915C0290915D0201967A
:1006200090935D0280935C0211500E949612F1CF6C
:10063000C0910601D09107018153883058F4C091D0
:100640000801D09109010E94B712BC01CE010E949D
:10065000C023EB017E01F694E7940E9496128E323D
:1006600061F480915C0290915D02019690935D022D
:1006700080935C02CE0DDF1DEECFFE018091530210
:10068000882349F0CE0196958795809352028091F8
:100690005202E81BF109C0910401D091050101113A
:1006A00004C01F3F11F0C11105C040E0BF0188EE3A
:1006B00093E046C0113130F020EF210F203618F0C2
:1006C0002FE501C020E0822F6CE00E94B423682F48
:1006D00074EF7603A0011124BA01620F711D9B0112
:1006E0006C30710540F4220F331FD901A65CBE4F58
:1006F0002D913C9102C020E030E0873081F0082E3F
:1007000002C0220F331F0A94E2F7823028F0C90199
:1007100005966AE070E00CC0C90190580CC0C90190
:1007200026E0880F991F2A95E1F7029665E070E0B0
:100730000E94C023CB014C2FC03108F04FE0BF0115
:100740000E94DF120AC06091520270E040E088EE21
:1007500093E00E94DF1210925202FF91EF91DF911D
:10076000CF91BF91AF919F918F917F916F915F9149
:100770004F913F912F911F910F91FF90EF90DF903C
:10078000CF90BF90AF909F908F907F906F900F9081
:100790000FBE0F901F9018951F920F920FB60F92D9
:1007A00011242F933F934F935F936F937F938F9376
:1007B0009F93AF93BF93EF93FF938091B900887F8E
:1007C000803609F49CC068F5883209F45BC090F467
:1007D000803109F454C038F4882309F4F6C0883015
:1007E00009F44DC0F6C0883109F44CC0803209F4D8
:1007F0005DC0EFC0803409F468C048F4803309F468
:1008000055C0883309F0E5C08093BA02D8C080355E
:1008100009F44FC0883509F45DC0883409F0D9C0A7
:10082000D6C0883909F4C7C0A8F4883709F467C06E
:1008300038F4883609F463C0803709F460C0C9C051
:10084000883809F4B8C0803909F45FC0803809F0ED
:10085000C0C05BC0803B09F486C038F4803A09F41C
:1008600066C0883A09F47FC0B4C0803C09F4A7C0D0
:10087000883C09F4A4C0883B09F48AC0AAC08091CE
:10088000970210C09091B9028091B802981770F544
:10089000E091B90281E08E0F8093B902F0E0E85652
:1008A000FD4F80818093BB0085EC86C08093BA02A7
:1008B0008EC0E091B90281E08E0F8093B9028091E1
:1008C000BB00F0E0E856FD4F80839091B902809123
:1008D000B8026EC0E091B90281E08E0F8093B90238
:1008E0008091BB00F0E0E856FD4F80838091BB0211
:1008F00081116DC081E08093960284EA61C083E03B
:100900008093BC0210925102CFCF8091510280326D
:1009100008F051C0E091510281E08E0F80935102A6
:100920008091BB00F0E0EF5CFD4F8083BDCF85EC94
:100930008093BC001092BC0280915102803230F44E
:10094000E0915102F0E0EF5CFD4F108260915102A6
:1009500070E0E0912F02F091300281E392E009957E
:100960001092510236C084E08093BC0210922E0295
:1009700010922D02E0912B02F0912C0209958091AA
:100980002D02811105C081E080932D0210920B028F
:10099000E0912E0281E08E0F80932E02F0E0E55F61
:1009A000FD4F80818093BB0090912E0280912D029B
:1009B000981708F479CF85E88093BC000AC085ECCD
:1009C0008093BC001092BC0204C01092BA020E9434
:1009D0000F01FF91EF91BF91AF919F918F917F9107
:1009E0006F915F914F913F912F910F900FBE0F909C
:1009F0001F90189580910602811105C081E08093B7
:100A000006020E940012F8948091600290916102A7
:100A1000789490930802809307026EE873E00E9436
:100A2000D4237093E4016093E30180910602811165
:100A300005C081E0809306020E940012F894809124
:100A40005E0290915F02789490930A02809309026B
:100A50006EE873E00E94D4237093E6016093E50191
:100A600008958F929F92AF92BF92CF92DF92EF92B2
:100A7000FF920F931F930E94E014E090DD03F0902B
:100A8000DE038091E1019091E201E81AF90AF09207
:100A90000502E09204020E945A0F2091DF0130917A
:100AA000E001AB01421B530B9A017093E00160938C
:100AB000DF01D7010E94EE2320E030E040EE50E05D
:100AC0000E94F523EDE8AE2EF8E3BF2EACE0CA2E6F
:100AD000DD24D394E12CF12C00E010E00E943124BD
:100AE00049015A018091EB019091EC01A091ED0137
:100AF000B091EE01880D991DAA1DBB1D8093EB01DD
:100B00009093EC01A093ED01B093EE019D01552768
:100B100037FD5095452FA8E6B1E00E948122BB2702
:100B200097FDB095AB2F8093E7019093E801A093D8
:100B3000E901B093EA011F910F91FF90EF90DF90D0
:100B4000CF90BF90AF909F908F900895CF93DF93F9
:100B500000D000D000D0CDB7DEB780912D048F3FFC
:100B600061F061E00E94F00E61E080912D040E942E
:100B7000750E8BE193E00197F1F7E0912004F0917D
:100B800021040190F081E02DBE016F5F7F4F80E274
:100B900094E009950E944D1889819A812091D9018C
:100BA0003091DA01821B930B9093F4018093F3014F
:100BB0008B819C812091DB013091DC01821B930BA6
:100BC0009093F6018093F5018D819E812091DD0146
:100BD0003091DE01821B930B9093F8018093F70113
:100BE00026960FB6F894DEBF0FBECDBFDF91CF9132
:100BF0000895CF92DF92EF92FF920F931F93CF93BE
:100C0000DF93CDB7DEB72C970FB6F894DEBF0FBEDB
:100C1000CDBF10E080913404181788F4E0913204BD
:100C2000F091330483E0189FE00DF11D11248081C1
:100C30008F3118F462E00E94F00E1F5FEBCF8091BD
:100C400035048F3170F460E00E94750E61E0809190
:100C500035040E94F00E80913D0490913E040E9464
:100C60004F0F8091360490913704892B01F58CE069
:100C7000EEE2F1E0DE01119601900D928A95E1F726
:100C80006CE070E080E090E00E940526009779F02B
:100C90002CE0FE013196DC0101900D922A95E1F7DE
:100CA000909337048093360486E080933804209133
:100CB00032043091330480E090913404891750F469
:100CC000F90193E0899FE00DF11D11241282118238
:100CD0008F5FF2CF10E080913804181708F07EC0C3
:100CE0009091360480913704E92FF82FE10FF11D20
:100CF000E10FF11DC080D1804091390450913A0438
:100D0000B60180E090E00E94D31180913B04909165
:100D10003C040E944F0F00E0809134040817E0F477
:100D200083E0089F70011124E0913204F0913304B4
:100D3000EE0DFF1D80818F3168F40E944C0E892BCF
:100D400049F4E0913204F0913304EE0DFF1D8181EE
:100D50008F5F81830F5FE0CF0E94B91180913D04C6
:100D600090913E040E944F0F4091390450913A04F3
:100D7000B60181E090E00E94D31180913B049091F4
:100D80003C040E944F0F00E0809134040817E0F407
:100D900093E0099F70011124E0913204F091330433
:100DA000EE0DFF1D80818F3168F40E944C0E892B5F
:100DB00049F4E0913204F0913304EE0DFF1D82817D
:100DC0008F5F82830F5FE0CF0E94B91180913D0455
:100DD00090913E040E944F0F1F5F7DCF84E10E94DF
:100DE000F81310913404811758F4E0913204F09113
:100DF000330493E0899FE00DF11D1124818101C02E
:100E000080E08093F90186E10E94F813811758F47D
:100E1000E0913204F091330493E0899FE00DF11DDD
:100E20001124818101C080E08093FA0186E10E9453
:100E3000F813811758F4E0913204F091330493E0F1
:100E4000899FE00DF11D1124828101C080E0809313
:100E5000FB0184E00E94F813811758F4E0913204FA
:100E6000F091330493E0899FE00DF11D11248281FC
:100E700001C080E08093FC012C960FB6F894DEBF91
:100E80000FBECDBFDF91CF911F910F91FF90EF90DB
:100E9000DF90CF9008950E9453102091F10130917E
:100EA000F201621B730B7093F0016093EF010895E0
:100EB000882311F0479A01C047983F9A08958F926E
:100EC0009F92AF92BF92CF92DF92EF92FF9280916A
:100ED000F3019091F40187599109893F9105F0F44C
:100EE00081E00E945807C0900001D0900101E0907D
:100EF0000201F0900301A701960160E070E088EC28
:100F000091E40E94FC220E946E234B015C01A70128
:100F1000960160E070E086ED92E426C08091F701D2
:100F20009091F8018B5A910987319140A0F581E0A9
:100F30000E945807C0900001D0900101E09002018A
:100F4000F0900301A701960160E070E088EC92E464
:100F50000E94FC220E946E234B015C01A7019601B6
:100F600060E070E088ED91E40E94FC220E946E2314
:100F7000DC01CB01B4010E946C1164E670E080E0FA
:100F800090E0FF90EF90DF90CF90BF90AF909F9058
:100F90008F900C947F0F8091F5019091F60185560A
:100FA0009109893F910508F05CC02898209A81E05A
:100FB00090E00E945E180E9453107093F2016093BB
:100FC000F1018091F3019091F4018639910594F03B
:100FD00064E670E080E090E00E947F0F80E090E0A7
:100FE000FF90EF90DF90CF90BF90AF909F908F9049
:100FF0000C945E188091F7019091F8018A3A91055E
:101000003CF70E944B070E94A605C0900001D090BB
:101010000101E0900201F0900301A701960160E058
:1010200070E088EC92EC0E94FC220E946E234B013F
:101030005C01A701960160E070E086ED92EC0E94F1
:10104000FC220E946E23DC01CB01B4010E946C11D2
:101050008091EF019091F001893B9B4008F4B1CF62
:10106000B7CF5D98559AC0900001D0900101E090F3
:101070000201F0900301A701960160E070E088ECA6
:1010800092E40E94FC220E946E234B015C01A701A6
:10109000960160E070E086ED92E40E94FC220E94DE
:1010A0006E23DC01CB01B401FF90EF90DF90CF9075
:1010B000BF90AF909F908F900C946C11409157020D
:1010C0005091580220915502309156024217530711
:1010D000B4F49091E8009570E1F39091E80092FDEE
:1010E00019C08093F10080915702909158020196A7
:1010F0008F739927892B19F48EEF8093E8008091E4
:10110000570290915802019690935802809357028B
:1011100081E0089580E00895DF92EF92FF920F93AF
:101120001F93CF93DF93D82E8A017B01E40EF51E27
:10113000EB01CE15DF0571F0D7FE03C0FE018491EF
:1011400001C088810E945E0821968111F2CF8FEF45
:101150009FEF01C0C801DF91CF911F910F91FF90C8
:10116000EF90DF900895615030F02091F100FC0184
:1011700020830196F8CF289884E680934004089550
:10118000CF92DF92EF92FF920F931F93CF93DF9353
:101190006C017A018B01C0E0D0E0CE15DF0589F04B
:1011A000D8016D918D01D601ED91FC910190F081F6
:1011B000E02DC6010995892B11F47E0102C021960C
:1011C000ECCFC701DF91CF911F910F91FF90EF906E
:1011D000DF90CF900895FC01538D448D252F30E092
:1011E000842F90E0821B930B541710F0CF96089534
:1011F00001970895FC01918D828D981761F0828D81
:10120000DF01A80FB11D5D968C91928D9F5F9F733A
:10121000928F90E008958FEF9FEF0895FC01918DDC
:10122000828D981731F0828DE80FF11D858D90E049
:1012300008958FEF9FEF0895FC01918D228D892FE6
:1012400090E0805C9F4F821B91098F7399270895CE
:1012500080EE92E00E941C0921E0892B09F420E035
:10126000822F0895FC01848DDF01A80FB11DA35AC0
:10127000BF4F2C91848D90E001968F739927848FB6
:10128000A689B7892C93A089B1898C9180648C93AD
:10129000938D848D981306C00288F389E02D808198
:1012A0008F7D80830895EF92FF920F931F93CF93CA
:1012B000DF93EC0181E0888F9B8D8C8D981305C0A6
:1012C000E889F989808185FD24C0F62E0B8D10E018
:1012D0000F5F1F4F0F731127E02E8C8DE8120CC08B
:1012E0000FB607FCFACFE889F989808185FFF5CF31
:1012F000CE010E943209F1CF8B8DFE01E80FF11D66
:10130000E35AFF4FF0820B8FEA89FB89808180626C
:1013100007C0EE89FF896083E889F989808180644C
:10132000808381E090E0DF91CF911F910F91FF903A
:10133000EF900895CF93DF93EC01888D8823C9F057
:10134000EA89FB89808185FD05C0A889B9898C91CE
:1013500086FD0FC00FB607FCF5CF808185FFF2CF69
:10136000A889B9898C9185FFEDCFCE010E94320901
:10137000E7CFDF91CF91089580E090E0892B29F0AD
:101380000E94280981110C9400000895CF93DF93E7
:101390001F92CDB7DEB76983DC01ED91FC9102802D
:1013A000F381E02D41E050E0BE016F5F7F4F099572
:1013B0000F90DF91CF91089583E08093E9008091B1
:1013C000F200882319F08AE38093E8000895FC0175
:1013D0008485958597FD0BC09FB7F89482E0809334
:1013E000E9008091F2009FBF90E0019608959FB7B9
:1013F000F89482E08093E9008091F2009FBF90E032
:10140000089590E0FC013197EF30F105B0F5EA5A0C
:10141000FF4F0C94E823809180008F7703C0809168
:1014200080008F7D80938000089580918000877F69
:10143000F9CF84B58F7702C084B58F7D84BD0895C0
:10144000809190008F7707C0809190008F7D03C0BE
:1014500080919000877F8093900008958091C000D4
:101460008F7703C08091C0008F7D8093C000089566
:101470008091C200877F8093C20008950E94CF268A
:101480000F931F93CF93DF931F92CDB7DEB782E008
:10149000898342E450E063E471E080E80E948C08B4
:1014A0000E942119DC0112960D911C9113970115D0
:1014B000110569F0D801ED91FC910280F381E02DD6
:1014C000BE016F5F7F4FC801099597FF07C08981F3
:1014D0000F90DF91CF911F910F910895F801008532
:1014E0001185E5CF8F929F92AF92BF92CF92DF92FC
:1014F000EF92FF920F931F93CF93DF935C016B01E9
:101500007A0180911801882309F45BC0809141041D
:10151000882309F456C08091D70180FF05C08091CF
:10152000E00082608093E000E70110E00AEF83E0D2
:10153000882E9AE3992E2097D9F10E9410198111D3
:101540000AC0015009F43DC061E070E080E090E025
:101550000E947F0FF0CF282F30E0C217D3070CF482
:101560008C2F4FB7F8948092E9009091E80095FF96
:101570001DC0282F30E0C21BD30BF601982F9150CD
:1015800020F081918093F100FACFC20ED31E112377
:1015900019F09092E80009C08091E80085FD06C02E
:1015A0009092E80011E0209709F010E04FBFC3CF00
:1015B0001111C3CF5D9884E6809359021E141F0455
:1015C00044F081E090E0F5019383828380E090E035
:1015D00001C0C701DF91CF911F910F91FF90EF9054
:1015E000DF90CF90BF90AF909F908F9008950E9412
:1015F000101990E00895CF93DF931F92CDB7DEB717
:10160000FC018485958597FD05C02FEF3FEF358759
:1016100024870BC0CE0101960E94E618019719F4A9
:10162000898190E002C08FEF9FEF0F90DF91CF9103
:1016300008950F931F93CF93DF931F92CDB7DEB71B
:101640008C01FC018485958597FF0EC0CE01019623
:101650000E94E618019719F4298130E002C02FEFAB
:101660003FEFF80135872487F801848595850F9031
:10167000DF91CF911F910F9108951F920F920FB696
:101680000F9211248F939F938091E1009091E1003C
:10169000937F9093E10083FF0FC01092E90091E0E7
:1016A0009093EB001092EC0092E39093ED00109277
:1016B000410498E09093F00082FF20C093E0909363
:1016C000E9009091F200992319F09AE39093E800D1
:1016D00090915902992339F0909159029150909329
:1016E0005902992389F190914004992339F09091FE
:1016F0004004915090934004992341F184FF10C01D
:101700008091E2008E7E81608093E2008091E10012
:101710008F7E8093E1008091D7018E7E806111C021
:1017200080FF16C08091E2008E7E80618093E2008F
:101730008091E1008E7E8093E1008091D7018E7EC2
:1017400081608093D70104C05D9ACDCF289AD6CF0F
:101750009F918F910F900FBE0F901F9018951F9221
:101760000F920FB60F921124CF92DF92EF92FF9259
:101770000F931F932F933F934F935F936F937F9399
:101780008F939F93AF93BF93EF93FF93CF93DF9389
:10179000CDB7DEB76C97DEBFCDBF1092E900809168
:1017A000E80083FFEDC168E0CE0145960E94B308D2
:1017B00082EF8093E8008D8987FF05C09091E80053
:1017C00090FFFCCF03C09EEF9093E800982F907697
:1017D00009F0C6C09E892F89188D91110CC08038E0
:1017E00029F48091D8018093F10002C01092F10099
:1017F0001092F10048C1422F50E0512B913051F42A
:10180000811141C14130510509F03DC18091D8019C
:101810008D7F0BC0933061F4811135C1413051058A
:1018200009F031C18091D80182608093D8012BC129
:10183000953041F48091E80080FFFCCF2068209330
:10184000E30021C1963009F05FC0EB8CFC8C109254
:10185000E9001092580210925702123091F510923E
:101860005602109255020E94400A99E0BE016F5F35
:101870007F4FDB01E92F1D92EA95E9F799831A83DF
:1018800091E09E8390EA98879AEF9987209157027A
:1018900030915802275F3F4F3C832B838D831092FA
:1018A000E9001092580210925702F0925602E0920C
:1018B000550249E050E080E00E948C080E94400AF6
:1018C000E2C0F0925602E09255020E942119DC011A
:1018D0001296ED90FC901397E114F10409F4C0C046
:1018E000D701ED91FC910480F581E02DBE016B5E86
:1018F0007F4FC7010995009719F00CF0C4C0C7C00D
:10190000F701E084F184E8CF973009F4C0C0983043
:1019100021F481E08093F100B6C0993009F0B3C0A2
:10192000837009F0B4C0E3E5F1E081E021E036E343
:101930009081992361F08093E9002093EB009191CD
:101940009093EC003093ED008F5F873089F78EE73E
:101950008093EA001092EA008F898093410493C03B
:101960008B8D9C8D1092E9001092580210925702B4
:101970009093560280935502898D811156C08E89AD
:101980009D89913A59F4813209F081C047E050E0D5
:1019900061E171E080E00E948C0875C0913209F02D
:1019A00076C0833289F4888D90E0982F88272F891C
:1019B000822BA0E0B0E080930D0190930E01A093E4
:1019C0000F01B09310015FC0803269F48091E8008C
:1019D00082FFFCCF67E081E191E00E94B3088BEFCA
:1019E0008093E80006C0823209F04DC08F89809351
:1019F00018018091D601882319F0EEEFFAE002C0B9
:101A0000E0E0F8E08091110190911201A0911301A2
:101A1000B0911401803B9440A105B10509F07BC051
:101A20008091180180FF93C076C00E942119DC01CB
:101A300012960D911C9113970115110541F1D801D2
:101A4000ED91FC910190F081E02DBE016B5E7F4F26
:101A5000C8010995811117C0F80100851185ECCFE7
:101A6000113009F44EC0133091F48F89882309F4A2
:101A700045C0823081F440E860E187EA91E00E944D
:101A8000D720882321F08EEF8093E80079C081E28F
:101A90008093EB0075C0813029F440E86BE08BE95E
:101AA00091E0EDCF833099F70E942119DC01129665
:101AB000ED90FC9013978E010F5F1F4F6801E114AA
:101AC000F10479F0D701ED91FC910680F781E02DCA
:101AD000B801C7010995080F111DF701E084F184D1
:101AE000EECFD8011C92F60101900020E9F7319762
:101AF000BF016C197D0940E0C601C1CF65E871E006
:101B000002C069E871E06115710509F2FB014491B9
:101B100050E080E840CF0FB6F894A895809160001F
:101B2000886180936000109260000FBEA895EE3F20
:101B30002AE0F20739F08091FE0A9091FF0A918322
:101B40008083A1CF1092FF0A1092FE0A9CCFEE3F35
:101B50008AE0F80731F0808191819093FF0A8093A9
:101B6000FE0A87E797E7918380839BE088E10FB6C1
:101B7000F894A895809360000FBE9093600083CF87
:101B80006C960FB6F894DEBF0FBECDBFDF91CF913C
:101B9000FF91EF91BF91AF919F918F917F916F9145
:101BA0005F914F913F912F911F910F91FF90EF9077
:101BB000DF90CF900F900FBE0F901F90189561157A
:101BC000710579F0FB0101900020E9F73197AF0131
:101BD000461B570BDC01ED91FC910280F381E02D57
:101BE000099480E090E008951F920F920FB60F9233
:101BF00011242F933F934F935F936F937F938F9312
:101C00009F93AF93BF93EF93FF9380EE92E00E9478
:101C10003209FF91EF91BF91AF919F918F917F9189
:101C20006F915F914F913F912F910F900FBE0F9049
:101C30001F9018951F920F920FB60F9211242F9399
:101C40008F939F93EF93FF93E091F002F091F10255
:101C50008081E091F602F091F70282FD12C090813E
:101C60008091F9028F5F8F732091FA02821751F0F1
:101C7000E091F902F0E0E052FD4F958F8093F90278
:101C800001C08081FF91EF919F918F912F910F90D3
:101C90000FBE0F901F901895CF93DF93282F30E041
:101CA000F901EC5DFE4F8491F901EB5FFE4FD49199
:101CB000F901EA51FF4FC491CC2391F081110E94A8
:101CC000010AEC2FF0E0EE0FFF1FE852FF4FA59145
:101CD000B491EC91ED2381E090E021F480E002C02A
:101CE00080E090E0DF91CF9108951F93CF93DF9331
:101CF000282F30E0F901EC5DFE4F8491F901EB5F94
:101D0000FE4FD491F901EA51FF4FC491CC23C9F0A1
:101D1000162F81110E94010AEC2FF0E0EE0FFF1F39
:101D2000E653FF4FA591B4918FB7F894111105C0F8
:101D30009C91ED2FE095E92302C0EC91ED2BEC9303
:101D40008FBFDF91CF911F91089508952E98269A05
:101D50002D98259A2A98229A2998219A80EA809388
:101D6000800081E18093810080E991E09093870079
:101D700080938600109289001092880010928B0048
:101D800010928A0008954FB141708CB186FB88276C
:101D900080F98427209166025091650260915E026D
:101DA00070915F02982F9227292F30E0942F95276A
:101DB000291B3109260F371F30935F0220935E02E3
:101DC0002091650290916602821729F0491719F057
:101DD00091E09093640280936502409366020895B7
:101DE000CF93DF9390E0FC01EB5FFE4F2491FC0169
:101DF000EA51FF4F8491882361F190E0880F991F89
:101E0000FC01E854FE4FC591D491FC01E653FF4F0D
:101E1000A591B491611109C09FB7F894888120956C
:101E200082238883EC912E230BC0623061F49FB72C
:101E3000F8943881822F809583238883EC912E2B10
:101E40002C939FBF06C08FB7F894E8812E2B288370
:101E50008FBFDF91CF910895CF93DF93EC018885F9
:101E600081110FC081E088878A85882311F062E0A4
:101E700001C060E089850E94F00E8FE090E001973C
:101E8000F1F789850E944C0E2B8530E041E08217E6
:101E9000930709F440E0842FDF91CF9108958230B9
:101EA000910538F0880F991F880F991F05970197A2
:101EB000F1F708953FB7F894809170029091710204
:101EC000A0917202B091730226B5A89B05C02F3F66
:101ED00019F00196A11DB11D3FBFBA2FA92F982F50
:101EE0008827820F911DA11DB11DBC01CD0142E0CB
:101EF000660F771F881F991F4A95D1F708958F9213
:101F00009F92AF92BF92CF92DF92EF92FF926B01BE
:101F10007C010E945A0F4B015C01C114D104E10401
:101F2000F104F1F00E945A0FDC01CB0188199909E4
:101F3000AA09BB09883E9340A105B10570F321E0D1
:101F4000C21AD108E108F10888EE880E83E0981ED5
:101F5000A11CB11CC114D104E104F10419F7DDCFB7
:101F6000FF90EF90DF90CF90BF90AF909F908F90B9
:101F700008957F928F929F92AF92BF92CF92DF92FD
:101F8000EF92FF920F931F93CF93DF93FC01228573
:101F90003385232B09F479C07B01EC01D12C8C858E
:101FA000D816F0F40D2D10E08E859F85F801EE0F08
:101FB000FF1FEE0DFF1D91838083EA85FB85E00FF7
:101FC000F11F61E080810E94750E8A859B85FC016E
:101FD000E00FF11F61E080810E94F00ED394DFCF0B
:101FE00083E290E00197F1F710E08C851817A8F4D0
:101FF000C12ED12CEA85FB85EC0DFD1D60E08081B2
:102000000E94F00E8A859B85FC01EC0DFD1D60E0B1
:1020100080810E94750E1F5FE8CF0E945A0F4B010E
:102020005C010E945A0FAB01BC01481959096A09A9
:102030007B098E859F85A0E0B0E0481759076A07A5
:102040007B0718F50E945A0F6B01C818D908712C2C
:102050008C85781630F7072D10E0EA85FB85E00FB8
:10206000F11F80810E944C0E892B51F4000F111F2B
:10207000F701E00FF11F80819181C816D90610F099
:102080007394E6CFD182C082FBCFDF91CF911F91B5
:102090000F91FF90EF90DF90CF90BF90AF909F9007
:1020A0008F907F9008952FB7F89460916C02709193
:1020B0006D0280916E0290916F022FBF08951F9262
:1020C0000F920FB60F9211242F933F938F939F93EC
:1020D000AF93BF9380916C0290916D02A0916E02BC
:1020E000B0916F0230916B0223E0230F2D3720F463
:1020F0000196A11DB11D05C026E8230F0296A11D62
:10210000B11D20936B0280936C0290936D02A0939B
:102110006E02B0936F028091700290917102A09153
:102120007202B09173020196A11DB11D80937002DD
:1021300090937102A0937202B0937302BF91AF911A
:102140009F918F913F912F910F900FBE0F901F90F5
:1021500018951F920F920FB60F9211242F933F9351
:102160004F935F936F937F938F939F93AF93BF939F
:10217000EF93FF93E0912201F09123010995FF91E4
:10218000EF91BF91AF919F918F917F916F915F91EF
:102190004F913F912F910F900FBE0F901F90189568
:1021A0001F920F920FB60F9211242F933F934F93CC
:1021B0005F936F937F938F939F93AF93BF93EF93AF
:1021C000FF93E0912001F09121010995FF91EF919A
:1021D000BF91AF919F918F917F916F915F914F913F
:1021E0003F912F910F900FBE0F901F9018951F9247
:1021F0000F920FB60F9211242F933F934F935F933B
:102200006F937F938F939F93AF93BF93EF93FF93BE
:10221000E0911E01F0911F010995FF91EF91BF918F
:10222000AF919F918F917F916F915F914F913F916E
:102230002F910F900FBE0F901F9018951F920F9225
:102240000FB60F9211242F933F934F935F936F9389
:102250007F938F939F93AF93BF93EF93FF93E091FF
:102260001C01F0911D010995FF91EF91BF91AF9174
:102270009F918F917F916F915F914F913F912F919E
:102280000F900FBE0F901F9018951F920F920FB6D0
:102290000F9211242F933F934F935F936F937F93EC
:1022A0008F939F93AF93BF93EF93FF93E0911A01A6
:1022B000F0911B010995FF91EF91BF91AF919F9113
:1022C0008F917F916F915F914F913F912F910F90DF
:1022D0000FBE0F901F9018950F931F93CF93DF930E
:1022E0008C01EB0180916A02811105C081E080932D
:1022F0006A020E94A60E17FF05C0119501951109EB
:1023000081E001C080E0013991E0190714F000E993
:1023100011E010938B0000938A00882311F02A9A11
:1023200001C02A98229A80916A02811105C081E039
:1023300080936A020E94A60ED7FF05C0D195C19571
:10234000D10981E001C080E0C13991E0D90714F0E2
:10235000C0E9D1E0D0938900C0938800882311F0B0
:10236000299A01C02998219ADF91CF911F910F914D
:10237000089546983E9AE0E9F0E082E0808310926A
:1023800091001092710010821092990010929800A2
:10239000109297001092960010929500109294005F
:1023A00086988E980895FC01109271009B01461743
:1023B000570708F49A0146983E9890E89093900049
:1023C00010929100909392003E9AEF2B11F08E9A0A
:1023D00001C08E98869A5093970040939600415082
:1023E00051095093950040939400309399002093A5
:1023F000980082E88093900089E18093910008958D
:1024000024982C9A6A98729A6E98769A8098889AEC
:1024100081E08093680090E190936B008BBB83EC2C
:102420009EE09093230180932201EAE6F0E0808110
:102430008F7C80618083EE9A8CB182FB882780F943
:102440008093690293B12091690294FB882780F9F7
:1024500082278093680210926102109260021092AB
:1024600067028FB18170809366029CB120916602F1
:1024700096FB882780F982278093650210925F027D
:1024800010925E021092640208951F920F920FB68E
:102490000F9211242F933F934F935F936F937F93EA
:1024A0008F939F938CB190E095958795959587959F
:1024B000482F417023B130E054E0359527955A9567
:1024C000E1F7822793278170209169025091680279
:1024D0006091600270916102982F9227292F30E05D
:1024E000942F9527291B3109260F371F309361023E
:1024F000209360022091680290916902821729F06E
:10250000491719F091E09093670280936802409315
:1025100069029F918F917F916F915F914F913F9150
:102520002F910F900FBE0F901F901895809163020E
:10253000E0915C02F0915D02882311F0849101C06A
:1025400080819FEB980F9A3110F4805E089580325D
:1025500069F420915C0230915D02A9014F5F5F4FE9
:1025600050935D0240935C02232B01F708951F9363
:10257000CF93DF930E949612C0E0D0E01AE090ED76
:10258000980F9A30B8F41C9F90011D9F300D1124B4
:10259000E901C80FD11D87FDDA95E09780915C02B3
:1025A00090915D02019690935D0280935C020E947F
:1025B0009612E5CFCE01DF91CF911F9108952F9212
:1025C0003F924F925F926F927F928F929F92AF92C3
:1025D000BF92CF92DF92EF92FF920F931F93CF9310
:1025E000DF93CDB7DEB727970FB6F894DEBF0FBEE7
:1025F000CDBF9F838E831B014D8380916202811129
:102600001BC081E080936202109272001092C000A1
:1026100094E09093C10099E09093C2008093C3002E
:1026200083E08093BF0088EE8093D1001092BF00BA
:102630001092D200579A7894109219012E813F81FE
:1026400037FF05C03F773F832E830AE001C001E0DA
:1026500088E2089F802D112490E04E815F81481709
:10266000590708F4C2C0013039F44131574220F013
:10267000E0E1F7E2FF83EE83802E912CA12CB12CB8
:102680008E819F81969587959C0140E050E029833B
:102690003A834B835C834E815F812A01612C712CCC
:1026A000A501940160E072E18AE790E00E94A42312
:1026B00029813A814B815C81620F731F841F951FB2
:1026C000A30192010E94622269017A01EE24FF2493
:1026D00010E01F5FC11434E0D306E104F10408F1F7
:1026E00020E032E14AE750E0012E04C055954795BD
:1026F000379527950A94D2F7C501B4010E94A42307
:1027000029813A814B815C81620F731F841F951F61
:10271000A30192010E94622269017A01EE24FF2442
:10272000D8CF0A3049F48E819F8105966AE070E027
:102730000E94C0237F836E834E815F81483E83E089
:10274000580759F09101DA010E94ED2228EE33E09A
:1027500040E050E00E9462221901109272008091C4
:10276000C100807F182B1093C100BB27AF2D9E2D79
:102770008D2D8093BF00C092D1002D81203108F0B3
:102780002FE080E190E0821B910904C0F694E79469
:10279000D794C7948A95D2F78D2D99278093BF003F
:1027A000C092D20030925B0220925A0289B38FEF1E
:1027B00089BB84E08093720027960FB6F894DEBF41
:1027C0000FBECDBFDF91CF911F910F91FF90EF9082
:1027D000DF90CF90BF90AF909F908F907F906F9041
:1027E0005F904F903F902F9008959F838E8344CFAA
:1027F00040913404209132043091330490E09417D6
:1028000049F02D5F3F4FF90133975081581721F060
:102810009F5FF5CF8FEF0895892F08952091DF02F4
:1028200090913F04213208F04AC08091BC0281118E
:10283000FCCF32E03093BC0231E03093BB023FEF7B
:102840003093BA021092B9022093B802AFEBB2E013
:1028500048E952E0FA013E2F341B321718F43D913B
:102860003193F9CF1092970220919702990F922BF2
:102870009093970290919602913061F41092960293
:10288000909197029093BB009091BC0093FDF8CF7C
:1028900095EC01C095EE9093BC009091BC029230F3
:1028A000E1F39091BA029F3F79F08091BA028032B1
:1028B00041F08091BA02803331F084E005C081E0BC
:1028C00003C082E001C083E01092BE021092DF02DA
:1028D0001092BD02089591E09093BD0280933F0451
:1028E0001092BE021092DF0208959091BC029111E5
:1028F000FCCF613208F060E291E09093BC029093CB
:10290000BB022FEF2093BA021092B902260F209338
:10291000B8029093970290919702880F892B809329
:10292000970280919602813061F410929602809114
:1029300097028093BB008091BC0083FDF8CF85ECAB
:1029400001C085EE8093BC008091BC028130E1F330
:102950008091B902861710F46091B902A8E9B2E03B
:1029600026E732E0F9018E2F821B861718F48D912D
:102970008193F9CF1092750260937402862F0895A7
:10298000CF93C82F0E946B146FE08DEC93E00E94F0
:102990009D010E940E1481110FC061E08C2F0E94D6
:1029A00075149091740280917502981729F08DEC3E
:1029B00093E0CF910C9451018FEF9FEFCF91089549
:1029C000BF92CF92DF92EF92FF920F931F93CF931C
:1029D000DF938091E2030E946B1468EA8DEC93E030
:1029E0000E949D010E940E1466E08091E2030E9405
:1029F00075140E9453107B018091740290E0209125
:102A00007502821B91090697ACF48091E3039091C3
:102A1000E403892B89F30E9453106E197F0980917A
:102A2000E3039091E4038617970730F781E08093E2
:102A3000E50333C08DEC93E00E945101C82E8DEC6C
:102A400093E00E945101B82E8DEC93E00E94510159
:102A5000E82E8DEC93E00E945101D82E8DEC93E08E
:102A60000E945101F82E8DEC93E00E9451011B2D24
:102A700000E00C291093DA030093D903DD2D20E048
:102A8000C22FCE29D093DC03C093DB03982F882775
:102A90008F299093DE038093DD03DF91CF911F9107
:102AA0000F91FF90EF90DF90CF90BF9008950F931C
:102AB0001F93CF93DF93082F162FC9EDD3E089859D
:102AC0000E946B14602F8DEC93E00E949D01612F9A
:102AD0008DEC93E00E949D010E940E148E83DF9185
:102AE000CF911F910F9108958BE60E94C0148F3FE4
:102AF0002FEF920781F48AE60E94C0148F3F2FEFD8
:102B0000920761F489E60E94C014833D910541F566
:102B100021E030E02DC021E030E002C020E030E0D4
:102B2000873D9105D1F081E090E09093E10380939F
:102B3000E0030197029738F42130310511F08AE65D
:102B400008C08BE606C02130310511F088E601C0CF
:102B500089E68093E20381E0089582E090E0E5CF8A
:102B600088E60E94C014833D910529F420E030E0FE
:102B700080E090E0DACF80E00895EF92FF920F932B
:102B80001F93CF93DF93809102040E946B14809176
:102B9000FF0390910004039731F460910704709152
:102BA0000804606804C060910504709106048DEC0F
:102BB00093E00E949D010E940E148093FE0366E044
:102BC000809102040E9475140E945310EB018091C1
:102BD000740290E020917502821B91090697ACF473
:102BE0008091110490911204892B89F30E94531053
:102BF0006C1B7D0B8091110490911204861797072E
:102C000030F781E08093130474C08091FF039091AA
:102C100000040397F9F48DEC93E00E945101182F02
:102C20008DEC93E00E945101E82E8DEC93E00E9420
:102C30005101D82F8DEC93E00E945101F82E8DECBC
:102C400093E00E945101C82F8DEC93E00E94510146
:102C5000082F39C08DEC93E00E945101E82E8DECD5
:102C600093E00E945101182F8091FF03909100047E
:102C7000892BA9F48DEC93E00E945101F82E8DEC84
:102C800093E00E945101D82F8DEC93E00E945101F6
:102C9000082F8DEC93E00E945101C82F14C08DECD9
:102CA00093E00E945101082F8DEC93E00E945101A6
:102CB000C82F8DEC93E00E945101F82E8DEC93E02B
:102CC0000E945101D82F212F30E03E293093ED038F
:102CD0002093EC032D2F30E03F293093EF03209316
:102CE000EE032C2F30E0C901902B9093F1038093D9
:102CF000F003DF91CF911F910F91FF90EF90089516
:102D00001F93CF93DF931F92CDB7DEB7182F698340
:102D10000E946B1469818DEC93E00E949D010E94DA
:102D20000E14811112C061E0812F0E9475149091E0
:102D3000740280917502981741F08DEC93E00F902A
:102D4000DF91CF911F910C9451018FEF9FEF0F9066
:102D5000DF91CF911F910895BF92CF92DF92EF92B2
:102D6000FF920F931F93CF93DF93809101040E94F2
:102D70006B1468EA8DEC93E00E949D010E940E1492
:102D80008093FE0366E0809101040E9475140E9406
:102D900053107B018091740290E020917502821B98
:102DA00091090697ACF48091110490911204892B3B
:102DB00089F30E9453106E197F098091110490913C
:102DC00012048617970730F781E08093130433C00D
:102DD0008DEC93E00E945101C82E8DEC93E00E948F
:102DE0005101B82E8DEC93E00E945101E82E8DEC3C
:102DF00093E00E945101D82E8DEC93E00E94510186
:102E0000F82E8DEC93E00E9451011B2D00E00C295F
:102E10001093E7030093E603DD2D20E0C22FCE29B7
:102E2000D093E903C093E803982F88278F299093C4
:102E3000EB038093EA03DF91CF911F910F91FF90F5
:102E4000EF90DF90CF90BF9008950F931F93CF9393
:102E5000DF93082F162FC6EED3E08C8D0E946B14E3
:102E6000602F8DEC93E00E949D01612F8DEC93E02B
:102E70000E949D010E940E14888FDF91CF911F91B7
:102E80000F9108950F931F93CF93DF93082F162F61
:102E9000C6EED3E08B8D0E946B14602F8DEC93E017
:102EA0000E949D01612F8DEC93E00E949D010E9484
:102EB0000E14888FDF91CF911F910F91089520916B
:102EC000FF03309100042330310511F0803210F4FB
:102ED0000C9425170C9442176FE070E08DE10E946E
:102EE00080168934910561F06FE070E08EE10E94F8
:102EF00080168934910509F0A2C020E030E002C0BC
:102F000021E030E083E090E0909300048093FF03A1
:102F10008230910539F589E1809301048EE1809337
:102F2000020483E090E0909306048093050484E01B
:102F300090E0909308048093070487E090E09093DA
:102F40000A048093090488E090E090930C04809335
:102F50000B0485E090E090930E0480930D0486E0CE
:102F600090E030C08330910599F1019709F45FC07A
:102F70002130310509F461C088E1809301048EE1BC
:102F80008093020483E090E090930604809305040C
:102F900084E090E0909308048093070485E090E03B
:102FA00090930A048093090486E090E090930C04C7
:102FB00080930B0487E090E090930E0480930D04BF
:102FC00088E090E09093100480930F0481E00895CE
:102FD0002130310511F08EE101C08DE180930204B2
:102FE0008093010488E090E09093080480930704A4
:102FF00089E090E090930604809305048AE090E0D5
:1030000090930C0480930B048BE090E090930A045F
:10301000809309048CE090E09093100480930F0457
:103020008DE090E090930E0480930D04CFCF21307B
:10303000310509F470CF88E16FCF89E19ECF60E25E
:1030400070E089E10E948016019661F06FE070E007
:103050008EE10E94801621E030E0CC97D9F080E02C
:1030600090E052CF60E270E088E10E948016019605
:1030700079F06FE070E08EE10E94801631E020E090
:10308000CC9709F030E0832F922F20E030E03CCF46
:1030900080E0089582E090E037CF80912D048F3F4B
:1030A00061F061E00E94F00E60E080912D040E94CA
:1030B000750E8BE193E00197F1F708958F929F923F
:1030C000AF92BF92CF92DF92EF92FF920F931F9336
:1030D000CF93DF93CDB7DEB7A1970FB6F894DEBFDD
:1030E0000FBECDBF6C01990FEE08FF08F7FE33C08D
:1030F000E091E002F091E1020190F081E02D6DE2BB
:1031000080EE92E009958C0122273327A9012C1922
:103110003D094E095F0919A2CE0181967C019AE012
:10312000892E912CA12CB12CCA01B901A5019401C1
:103130000E94CB22605DF70162937F01211531056A
:103140004105510589F7BF0180EE92E00E94DF0D35
:10315000080F191F20C0A701960119A28E010F5D4B
:103160001F4F8AE0C82ED12CE12CF12CCA01B901E5
:10317000A70196010E94CB22605DF80162938F0146
:10318000211531054105510589F7BF0180EE92E017
:103190000E94DF0D8C0163ED71E080EE92E00E94F1
:1031A000DF0D800F911FA1960FB6F894DEBF0FBE02
:1031B000CDBFDF91CF911F910F91FF90EF90DF90E6
:1031C000CF90BF90AF909F908F900895FC01809119
:1031D0004104811103C08FEF9FEF08959FB7F894CA
:1031E00082E08093E9002091F20030E0121613068D
:1031F00014F421E030E02115310559F0289884E6D7
:10320000809340048091F10080838091F2008823B4
:1032100019F09FBFC90108958BE68093E800F9CFAC
:103220002FB7F89483E08093E9009091E800892F0C
:10323000807295FF04C09091F20080E4891B2FBF3B
:1032400008958091460481110DC082E0809342046C
:1032500084E080934304109245041092440481E07A
:103260008093460482E494E00895CF93DF93CDB732
:10327000DEB7C456D1090FB6F894DEBF0FBECDBF7E
:10328000789484B5826084BD84B5816084BD85B541
:10329000826085BD85B5816085BD80916E0081604D
:1032A00080936E00109281008091810082608093F3
:1032B00081008091810081608093810080918000F5
:1032C0008160809380008091910082608093910062
:1032D0008091910081608093910080919000816045
:1032E000809390008091C10084608093C1008091A0
:1032F000C10082608093C1008091C1008160809391
:10330000C1008091C30081608093C3008091C000A0
:1033100082608093C0008091C20081608093C2006F
:1033200080917A00846080937A0080917A00826034
:1033300080937A0080917A00816080937A008091F6
:103340007A00806880937A00109241041092D8012C
:103350001092D7018091D70081608093D70080EAD6
:103360008093D80089B5806189BD89B5826089BDA7
:1033700009B400FEFDCF61E070E080E090E00E94C3
:103380007F0F8091D8008F7C80618093D8008091DE
:10339000E000807F8093E0008091E1008E7E80934A
:1033A000E1008DE08093E200559A209AEEEFFFE76E
:1033B000859194918B3F9C4D19F481E08093D601C7
:1033C000E091F002F091F10282E08083E091EC0262
:1033D000F091ED021082E091EE02F091EF028FEC9D
:1033E00080831092F802E091F402F091F50286E0F9
:1033F0008083E091F202F091F3028081806180830A
:10340000E091F202F091F302808188608083E09184
:10341000F202F091F302808180688083E091F202F1
:10342000F091F30280818F7D80838AE090E0A0E0BC
:10343000B0E08093E4029093E502A093E602B0939B
:10344000E70280EE92E00E941C09892B61F063EB99
:1034500071E08DE793E00E94DF0D63ED71E08DE791
:1034600093E00E94DF0D1092750210927402109288
:10347000BE021092DF021092BC0281E08093BB0278
:103480001092960261E082E00E94750E61E083E096
:103490000E94750E8091B9008E7F8093B900809153
:1034A000B9008D7F8093B90088E48093B80085E4EB
:1034B0008093BC0064EF71E080E090E00E947F0F99
:1034C0008BE08093350469E070E080913204909144
:1034D00033040E940526FC01009769F090933304A1
:1034E0008093320483E08093340484E1808386E116
:1034F000838384E0868381E00E94580782E1898388
:1035000085E18A838CE08B8310922304109222043D
:10351000109225041092240410922704109226047D
:103520001092290410922804109231041092300451
:1035300083E080932C0480912A0490912B04892BA2
:1035400011F080E00BC083E090E00E94D8249093BB
:103550002B0480932A04892BA1F719C090912C0485
:10356000891790F4282F30E0E0912A04F0912B0481
:10357000E20FF31FA1E0B0E0AC0FBD1FA20FB31F1D
:103580009C9190838F5FEACF8BE080932D0480ED38
:1035900097E090932F0480932E04809124049091BF
:1035A0002504892B39F08091220490912304892BE2
:1035B000D1F420C000912C0410E0C801880F991F9D
:1035C0000E94D8249093250480932404009709F442
:1035D000BCC0FC0180E090E08017910724F71192B5
:1035E00011920196F9CF00E010E04BE1842E43E008
:1035F000942E1BC000912C0410E0C801880F991F65
:103600000E94D8249093230480932204009709F405
:103610009CC0FC0180E090E020ED37E0801791072E
:1036200014F7219331930196F9CF80912D048F3FA8
:1036300059F061E00E94F00E61E080912D040E943B
:10364000750EC4010197F1F7E0912004F091210477
:103650000190F081E02DBE016F5B7F4F80E294E02E
:1036600009950E944D18A0902C04B12CBE016F5FEB
:103670007F4FFE01EF5BFF4FAE014F5D5F4FCA0111
:103680003B0120E030E02A153B054CF50115110502
:1036900089F0DC01CD90DC90E080F180CE14DF0475
:1036A00048F0D301CD90DC90E080F180EC14FD0473
:1036B00048F00DC0E080F180DC01ED92FC92011534
:1036C000110579F7E080F180D301ED92FC922F5F34
:1036D0003F4FB2E06B0E711C32960296D4CF0F5F53
:1036E0001F4F0A30110509F0A0CFE0902204F0909E
:1036F0002304A0912404B091250420E030E08091BF
:103700002C0490E02817390704F5FB018191919171
:10371000BF010D911C9111970817190718F4119604
:103720009C938E93FA0181919191AF01F7010081F1
:1037300011818017910710F4918380832F5F3F4F91
:10374000F2E0EF0EF11C1296DACF80E00E945807EB
:1037500080EF90E09093DA018093D90188E790E0C0
:103760009093DC018093DB018CED90E09093DE017F
:103770008093DD0181E00E9458070E9474150E9429
:103780007415811109C02898209A68EE73E080E0D2
:1037900090E00E947F0FF9CF6FEF80E20E945715F3
:1037A00060E283E20E94571560E084E20E945715B0
:1037B00000E014E0C12CD12C76018091E2030E943C
:1037C0006B1467E28DEC93E00E949D010E940E1441
:1037D0008093DF0361E08091E2030E9475148DEC19
:1037E00093E00E9451010E940E140E94E014809107
:1037F000DD039091DE03092E000CAA0BBB0BC80E53
:10380000D91EEA1EFB1E01501109B9F6C701B60107
:1038100020E034E040E050E00E9462223093E20178
:103820002093E1010E945A0F7093E0016093DF0141
:1038300080E00E94580781E00E9458070E946C17A0
:103840000E946C17811109C02898209A68EE73E0D5
:1038500080E090E00E947F0FF9CF8091FF0390916C
:10386000000483309105A9F460E081E20E945F17B3
:1038700067E580E20E945F1764E684E20E945F17BA
:1038800060E285E20E945F1760E086E20E945F17B7
:103890001CC0029731F468E083E20E94421767E49B
:1038A00005C060E083E20E94421767E280E20E9466
:1038B00042176CE080E00E94251760E281E00E94E0
:1038C000251760E082E00E94251700E014E060E028
:1038D00070E0CB01A2966FAFA297A3967FAFA3979C
:1038E000A4968FAFA497A5969FAFA5970E94AC16FC
:1038F0000E94BD15C090E603D090E7030D2C000C8C
:10390000EE08FF08A2966FADA297A3967FADA3978E
:10391000A4968FADA497A5969FADA5976C0D7D1D20
:103920008E1D9F1D01501109A9F620E034E040E0F2
:1039300050E00E9462223093FE012093FD0180E05E
:103940000E9458075D98559AE0911404F09115046F
:103950000190F081E02D84E194E009958823A1F3A2
:103960006AE070E080E090E00E947F0FE091140434
:10397000F09115040190F081E02D84E194E0099527
:10398000882311F3E0911404F09115040190F08163
:10399000E02D84E194E009958111F4CF6AE070E0B4
:1039A00080E090E00E947F0FE0911404F0911504F4
:1039B0000190F081E02D84E194E009958111E2CF3E
:1039C0000E945310611571058105910511F00E9447
:1039D000082264EF71E080E090E00E947F0F3324C2
:1039E0003394812C912C80E8A82E8FE3B82E92E09E
:1039F000492E512C612C712CC12CD12CE12C20E4AE
:103A0000F22E5D9A559A80E00E945807289A209AD3
:103A10000E94A6050E94F9050E94FA040E94310541
:103A20000E94AC160E94BD150091E6031091E703B9
:103A30008091FD019091FE01081B190B109300026B
:103A40000093FF010E944B0780EE92E00E941C0948
:103A50001816190644F480EE92E00E94FA0890933A
:103A6000030280930202809102029091030281334B
:103A7000910519F43092010204C0C09711F410921C
:103A80000102809101028823E9F1C0920001D092E5
:103A90000101E0920201F0920301093E1340B4F4E7
:103AA0008091FA01863091F08091FB01863071F0AF
:103AB0008091F3019091F401813991403CF480911F
:103AC000F7019091F801833C9140CCF060E070E008
:103AD00080E090E063C18091F3019091F4018159FD
:103AE00091408735924008F45CC18091F701909134
:103AF000F801835C91408532924008F452C10E94E3
:103B00005F079EC18092000190920101A092020184
:103B1000B09203018091FB018630E9F681E090E0EC
:103B20000E945E1881E00E9458071092EB011092EB
:103B3000EC011092ED011092EE011092E70110924B
:103B4000E8011092E9011092EA010E94310580918A
:103B5000E7019091E801A091E901B091EA018D9708
:103B6000A105B1059CF40E9431050E94A60564E6FA
:103B700070E08BE190E00E946C118091F7019091D0
:103B8000F8018B5A91098731914008F70E94A605E8
:103B90008091F7019091F8018A3A91054CF40E94C6
:103BA000A60564E670E08BE690E00E946C11F0CF11
:103BB0000E9431058091E7019091E801A091E9010F
:103BC000B091EA010B97A105B1051CF10E943105E6
:103BD0000E94A6058091F3019091F4018759910903
:103BE000893F910518F460E070E00EC08091F70104
:103BF0009091F8018B5A91098731914018F464E64D
:103C000070E002C069E170E08BE690E00E946C1108
:103C1000D1CF64E670E08BE690E00E946C110E94C8
:103C2000F9050E9453107093F2016093F1018091A5
:103C3000FC01863080F48091EF019091F001883B87
:103C40009B4048F40E944B070E94F9050E94A6057C
:103C50000E945F07ECCF0E94F9058091FC0186303D
:103C600039F40E94F9050E94A6050E945F07F5CF6E
:103C70000E9453107093F2016093F1010E944B0770
:103C80008091EF019091F001883B9B4038F40E94B5
:103C90004B070E94A6050E945F07F2CF1092EB012E
:103CA0001092EC011092ED011092EE011092E701DA
:103CB0001092E8011092E9011092EA010E94310588
:103CC0008091E7019091E801A091E901B091EA01AA
:103CD000843D9F4FAF4FBF4F9CF00E9431050E9423
:103CE000A60569E170E08BE690E00E946C1180917E
:103CF000F3019091F40187599109893F910500F7EB
:103D00000E94A6058091F3019091F40186399105F6
:103D10004CF40E94A60564E670E08BE690E00E94F9
:103D20006C11F0CF0E9431058091E7019091E8017C
:103D3000A091E901B091EA01863F9F4FAF4FBF4F7D
:103D40002CF50E9431050E94A6058091F701909103
:103D5000F8018B5A91098731914028F464E670E0AC
:103D600080E090E010C08091F3019091F4018759B8
:103D7000910964E670E0893F910518F48BE690E0C4
:103D800002C08BE190E00E946C11CECF80E090E009
:103D90000E945E1864E670E08BE690E00E946C1171
:103DA0004FC081E00E94580781E090E00E945E18B9
:103DB0000E94A60581E02091F3013091F4012139A0
:103DC00031400CF480E02091F7013091F801233C60
:103DD00031400CF056C037C00E94A6058091F30117
:103DE0009091F401863991050CF47EC01092EB019C
:103DF0001092EC011092ED011092EE011092E70189
:103E00001092E8011092E9011092EA010E94310536
:103E10008091E7019091E801A091E901B091EA0158
:103E20008A359105A105B1050CF46FC064E670E018
:103E30008BE690E00E946C1180E090E00E945E189A
:103E40000E94BC09DECD81110AC164E670E08BE6F8
:103E500090E00E946C110E9453107093F2016093E5
:103E6000F1010E944B078091EF019091F001883E93
:103E7000934010F70E944B070E94A6050E945F071F
:103E8000F2CF882309F469C00E940322A3019201A2
:103E90000E946222DC01CB010196A11DB11D81307F
:103EA0009105A105B10509F055C06EE670E08BE6FD
:103EB00090E00E946C110E9453107093F201609385
:103EC000F1010E944B078091EF019091F0018C323B
:103ED000914008F081CF0E944B076EE670E08BE6C0
:103EE00090E00E946C11EFCF8091F7019091F80162
:103EF0008A3A91050CF07ACF0E94A60564E670E03C
:103F00008BE690E00E946C1169CF0E9431050E94FF
:103F1000A6058091F7019091F8018B5A910987319C
:103F2000914028F464E670E080E090E010C0809159
:103F3000F3019091F4018759910964E670E0893F9B
:103F4000910518F48BE690E002C08BE190E00E94AE
:103F50006C115ECF823009F078CF1092EB01109295
:103F6000EC011092ED011092EE011092E701109217
:103F7000E8011092E9011092EA011092E401109216
:103F8000E3010E9431058091E7019091E801A09141
:103F9000E901B091EA01893D9F4FAF4FBF4F94F0C7
:103FA0000E9431050E94FA040E94A60569E170E0B2
:103FB0008BE690E00E946C118091E3019091E40106
:103FC00002974CF00E9431050E9453107093F20149
:103FD0006093F10127C08091F3019091F40187591A
:103FE0009109893F910578F6EDCF0E944B070E9419
:103FF00031050E94A6058091EF019091F001893B67
:104000009B4008F019CF8091F3019091F4018759FA
:104010009109893F9105A0F460E070E08BE690E0A3
:104020000E946C118091E7019091E801A091E90153
:10403000B091EA018C3A9F4FAF4FBF4FB4F6FCCE20
:104040008091F7019091F8018B5A91098731914045
:1040500018F462E370E0E2CF69E170E0DFCF109224
:10406000EB011092EC011092ED011092EE01109212
:10407000E7011092E8011092E9011092EA01109212
:10408000E6011092E5010E9431058091E7019091CF
:10409000E801A091E901B091EA018897A105B10575
:1040A00084F40E9431050E94FA0464E670E08BE11A
:1040B00090E00E946C118091E5019091E6010297D9
:1040C00024F31092E6011092E5010E9431058091DF
:1040D000E7019091E801A091E901B091EA018535ED
:1040E0009105A105B10584F40E9431050E94FA04EE
:1040F00064E670E08BE190E00E946C118091E50134
:104100009091E60102971CF364E670E08BE690E084
:104110000E946C110E9453107093F2016093F101A0
:104120000E944B078091EF019091F001883E9340EF
:1041300008F082CE0E944B070E94A6058091F701ED
:104140009091F8018B5A91098731914058F774CEBC
:104150008BEA91E0909321048093200480912A04BB
:1041600090912B04009711F00E946D2580912404FA
:1041700090912504009711F00E946D2580912804EC
:1041800090912904009711F00E946D2580912204DE
:1041900090912304009711F00E946D2580912604D0
:1041A00090912704009711F00C946D250895CF92FB
:1041B000DF92EF92FF920F931F93CF93DF931F92A3
:1041C000CDB7DEB7182F062FE42E862F880F8E5F0F
:1041D00099830E945E0883E00E945E08F12EC12E42
:1041E0009981D92E8C2D8F19801798F4F601E7FE4E
:1041F00002C0849101C080810E945E08182F80E077
:104200000E945E088123FFEFCF1ADF0A8111EACFF7
:1042100001C081E00F90DF91CF911F910F91FF902E
:10422000EF90DF90CF900895E0EEF2E013821282DB
:1042300088EE93E0A0E0B0E084839583A683B78303
:1042400029E631E0318320832DEC30E03587248767
:104250002CEC30E03787268728EC30E0318B208B40
:1042600029EC30E0338B228B2AEC30E0358B248B29
:104270002EEC30E0378B268B118E128E138E148E1F
:10428000EDE7F3E01382128284839583A683B783DC
:104290002BE731E0318320832FEF3FEF35872487F1
:1042A000EDECF3E01382128284839583A683B783B7
:1042B0008DE891E091838083E2E3F4E01182108243
:1042C00012828FEF838315821482168285EA91E031
:1042D0009287818782E492E09487838784EA91E0E1
:1042E00090878783E0E2F4E01382128215821482C1
:1042F00017821682118610861386128681EB91E052
:1043000091838083E4E1F4E01282158210868EE0CE
:10431000818781E0828783878FE991E09183808321
:1043200086E0E9E5F1E0A8EFB3E001900D928A950F
:10433000E1F786E0EFE5F1E0A2EFB3E001900D9246
:104340008A95E1F7E6EEF3E084E090E0928F818FCA
:1043500014A613A615A6E9EDF3E083E090E090879C
:10436000878313861286148608958F929F92AF9248
:10437000BF92CF92DF92EF92FF92CF93DF93EC0147
:10438000688179818A819B8161157105810591051B
:1043900021F464E279ED8BE597E02DE133EF41E024
:1043A00050E00E94622249015A019B01AC01A7EA38
:1043B000B1E40E9481226B017C01ACEEB4EFA50157
:1043C00094010E948F22DC01CB018C0D9D1DAE1D3E
:1043D000BF1DB7FF03C00197A109B0488883998327
:1043E000AA83BB83BC01CD019F77DF91CF91FF9062
:1043F000EF90DF90CF90BF90AF909F908F900895F7
:104400000E94B521089584E291E00E94B5210895AB
:1044100060932401709325018093260190932701D6
:10442000089597F99F6780E870E060E008959FEF36
:1044300080EC089500240A9416161706180609063B
:10444000089500240A94121613061406050608950A
:10445000092E0394000C11F4882352F0BB0F40F492
:10446000BF2B11F460FF04C06F5F7F4F8F4F9F4FD2
:10447000089557FD9058440F551F59F05F3F71F054
:104480004795880F97FB991F61F09F3F79F08795BB
:104490000895121613061406551FF2CF4695F1DF44
:1044A00008C0161617061806991FF1CF86957105D4
:1044B000610508940895E894BB2766277727CB0108
:1044C00097F90895052E97FB1EF400940E94792217
:1044D00057FD07D00E94CB2207FC03D04EF40C946A
:1044E000792250954095309521953F4F4F4F5F4F22
:1044F000089590958095709561957F4F8F4F9F4F50
:1045000008950E94ED22A59F900DB49F900DA49F49
:10451000800D911D11240895B7FF0C9481220E94F3
:104520008122821B930B08952F923F924F925F92AC
:104530006F927F928F929F92AF92BF92CF92DF92B3
:10454000EF92FF920F931F93CF93DF93CDB7DEB718
:10455000CA1BDB0B0FB6F894DEBF0FBECDBF0994AC
:104560002A88398848885F846E847D848C849B8403
:10457000AA84B984C884DF80EE80FD800C811B8111
:10458000AA81B981CE0FD11D0FB6F894DEBF0FBE40
:10459000CDBFED010895A1E21A2EAA1BBB1BFD01A0
:1045A0000DC0AA1FBB1FEE1FFF1FA217B307E40712
:1045B000F50720F0A21BB30BE40BF50B661F771F6A
:1045C000881F991F1A9469F760957095809590954A
:1045D0009B01AC01BD01CF010895A29FB001B39F23
:1045E000C001A39F700D811D1124911DB29F700DFC
:1045F000811D1124911D08950E9410230C942822DE
:104600000E94212258F00E941A2240F029F45F3FB4
:1046100029F00C94112251110C945C220C94172255
:104620000E94392268F39923B1F3552391F3951B26
:10463000550BBB27AA2762177307840738F09F5FC3
:104640005F4F220F331F441FAA1FA9F335D00E2E30
:104650003AF0E0E832D091505040E695001CCAF79D
:104660002BD0FE2F29D0660F771F881FBB1F261760
:1046700037074807AB07B0E809F0BB0B802DBF0137
:10468000FF2793585F4F3AF09E3F510578F00C9406
:1046900011220C945C225F3FE4F3983ED4F386959C
:1046A00077956795B795F7959F5FC9F7880F911D27
:1046B0009695879597F90895E1E0660F771F881F13
:1046C000BB1F621773078407BA0720F0621B730BC6
:1046D000840BBA0BEE1F88F7E09508950E947523AE
:1046E0006894B1110C945C2208950E94412288F0D4
:1046F0009F5798F0B92F9927B751B0F0E1F0660FA6
:10470000771F881F991F1AF0BA95C9F714C0B130E6
:1047100091F00E945B22B1E008950C945B22672F18
:10472000782F8827B85F39F0B93FCCF38695779515
:104730006795B395D9F73EF49095809570956195FE
:104740007F4F8F4F9F4F0895DB018F939F930E9460
:104750008122BF91AF91A29F800D911DA39F900DCB
:10476000B29F900D11240895991B79E004C0991F00
:10477000961708F0961B881F7A95C9F780950895BB
:10478000AA1BBB1B51E107C0AA1FBB1FA617B70777
:1047900010F0A61BB70B881F991F5A95A9F7809593
:1047A0009095BC01CD01089597FB072E16F4009457
:1047B00007D077FD09D00E94C02307FC05D03EF446
:1047C000909581959F4F0895709561957F4F0895BD
:1047D000EE0FFF1F0590F491E02D09940E94ED2249
:1047E000B7FF0895821B930B089597FB57FF0C9416
:1047F00005249F938F930E9405246E1B7F0BAF911E
:10480000BF918A0B9B0B0895E894DF93CF93FC0133
:10481000DB010E94ED227F936F93E9019A01AC01C5
:10482000BF93AF933F932F93DF010E94ED2226F4B5
:104830006C1B7D0B820B930B9E01EB01FC010E9414
:10484000CF24AF91BF912F913F910E94CF24BE0101
:10485000CF01F9012F913F91CF91DF910895689495
:1048600001C0E894F92FF12B12F00C946324A0E01E
:10487000B0E0EDE3F4E20C949A22092E059422F4C0
:104880000E94BF24112392F4F0E80F26FFEFE0947A
:10489000F09400951095B094C094D094A194BF0A60
:1048A000CF0ADF0AEF0AFF0A0F0B1F0B0E946E24CC
:1048B00007FC0E94BF24CDB7DEB7ECE00C94B62213
:1048C000689401C0E8948F929F92CF93DF930E94E7
:1048D0006E24DF91CF919F908F9008958824992422
:1048E000F401E401B0E49F93AA279A158B049C0479
:1048F000ED05FE05CF05D007A10798F4AD2FDC2FFD
:10490000CF2FFE2FE92D982C892E982F872F762FC9
:10491000652F542F432F322F2227B85031F7BF91E4
:1049200027C01B2EBF91BB27220F331F441F551FCB
:10493000661F771F881F991F881C991CEE1FFF1F79
:10494000CC1FDD1FAA1FBB1F8A149B04EC05FD05AD
:10495000CE05DF05A007B10748F08A189B08EC09CF
:10496000FD09CE09DF09A00BB10B21601A94E1F615
:104970002EF49401AF01BE01CD01000C08956095A5
:1049800070958095909530954095509521953F4F25
:104990004F4F5F4F6F4F7F4F8F4F9F4F08950E9434
:1049A000ED22460F571FC81FD91F08F431960895EE
:1049B000CF93DF938230910510F482E090E0E09194
:1049C0005004F091510420E030E0C0E0D0E0309796
:1049D00011F14081518148175907C0F04817590714
:1049E00061F482819381209719F09B838A832BC085
:1049F000909351048093500426C02115310519F07D
:104A00004217530718F49A01BE01DF01EF0102803B
:104A1000F381E02DDCCF2115310509F1281B390B7D
:104A20002430310590F412968D919C911397611565
:104A3000710521F0FB019383828304C0909351049C
:104A400080935004FD01329644C0FD01E20FF31F34
:104A500081939193225031092D933C933AC0209138
:104A60004E0430914F04232B41F420912A013091C0
:104A70002B0130934F0420934E0420912801309154
:104A800029012115310541F42DB73EB740912C0184
:104A900050912D01241B350BE0914E04F0914F04F1
:104AA000E217F307A0F42E1B3F0B2817390778F005
:104AB000AC014E5F5F4F2417350748F04E0F5F1F64
:104AC00050934F0440934E048193919302C0E0E0D1
:104AD000F0E0CF01DF91CF9108950F931F93CF9313
:104AE000DF93009709F48CC0FC0132971382128285
:104AF00000915004109151040115110581F4208199
:104B00003181820F931F20914E0430914F0428175A
:104B1000390779F5F0934F04E0934E0471C0D80142
:104B200040E050E0AE17BF0750F412962D913C9133
:104B30001397AD012115310509F1D901F3CF9D017D
:104B4000DA013383228360817181860F971F821778
:104B5000930769F4EC0128813981260F371F2E5FF6
:104B60003F4F318320838A819B8193838283452BAE
:104B700029F4F0935104E093500442C01396FC933F
:104B8000EE931297ED01499159919E01240F351F23
:104B9000E217F30771F480819181840F951F0296CB
:104BA00011969C938E938281938113969C938E93FE
:104BB0001297E0E0F0E0D80112968D919C91139746
:104BC000009719F0F8018C01F6CF8D919C91980116
:104BD0002E5F3F4F820F931F20914E0430914F0460
:104BE0002817390769F4309729F41092510410926C
:104BF000500402C01382128210934F0400934E049B
:104C0000DF91CF911F910F910895A0E0B0E0EBE00C
:104C1000F6E20C949822EC01009721F4CB010E945B
:104C2000D824B8C0FC01E60FF71F9C0122503109BF
:104C3000E217F30708F4ACC0D9010D911C9111974C
:104C400006171707B0F00530110508F49FC0C8011A
:104C500004978617970708F499C002501109061B9C
:104C6000170B019311936D937C93CF010E946D25D7
:104C70008DC05B01A01AB10A4C01800E911EA0915B
:104C80005004B091510440E050E0E12CF12C109719
:104C900009F44AC0A815B905D1F56D907C9011971B
:104CA000630182E0C80ED11CCA14DB0480F1A301A9
:104CB0004A195B096A0182E0C80ED11C1296BC90A9
:104CC00012971396AC91B5E0CB16D10440F0B282A6
:104CD000A38351834083D9016D937C930AC00E5FF7
:104CE0001F4FC301800F911FF90191838083EB2D2A
:104CF000FA2FE114F10431F0D7011396FC93EE93EF
:104D0000129744C0F0935104E09350043FC08D913A
:104D10009C9111974817590708F4AC017D01129630
:104D20000D90BC91A02DB3CF80914E0490914F0473
:104D300088159905E1F446175707C8F480912801B2
:104D400090912901009741F48DB79EB740912C01B5
:104D500050912D01841B950BE817F907C8F4F093C7
:104D60004F04E0934E04F901718360830FC0CB01BF
:104D70000E94D8247C01009759F0A801BE010E942E
:104D8000D426CE010E946D25C70104C0CE0102C009
:104D900080E090E0CDB7DEB7EEE00C94B42281E085
:104DA00090E0F8940C94DD26FB01DC0102C0019038
:104DB0000D9241505040D8F7089510E0C4EED0E075
:104DC00004C0FE010E94E8232196C53ED107C9F721
:044DD000F894FFCF85
:104DD4000000803F0F00F401D007040004FFFFFF30
:104DE400FF00E100000000000001A50EA50EA50EC5
:104DF400A50EA50E0100000000005204800004006E
:104E04000F0020003700550078009C01B501CF0148
:104E1400EA0107022602470269028E02B502DE0297
:104E24000A0300C18081000000018001800180FF2D
:104E34007FFF7FFF7F000000005309C008EB089A42
:104E4400091C09FA080E0900000000C609720AF7D5
:104E54000ADC09E709FB0A190B000000009D016D3B
:104E640001CD014101650151014201000000002C06
:104E74000F00000000B90F000000003E0A0000000F
:104E840000B90F426C7565746F6F746876657262F1
:104E9400696E64756E672068657267657374656CA6
:064EA4006C74000D0A0011
:2070000055C000006EC000006CC000006AC0000068C0000066C0000064C0000062C0000043
:2070200060C000005EC00000F2C400005AC0000058C0000056C0000054C0000052C00000EE
:2070400050C0000078C000004CC000004AC0000048C0000046C0000044C0000042C00000BE
:2070600040C000003EC000003CC000003AC0000038C0000036C0000034C0000032C0000048
:2070800030C000002EC000002CC000002AC0000028C0000026C0000024C0000022C00000A8
:2070A00020C000001EC000001CC0000011241FBECFEFDAE0DEBFCDBF11E0A0E0B1E0E2E3BC
:2070C000FFE702C005900D92A83AB107D9F711E0A8EAB1E001C01D92AE3BB107E1F78FD30B
:2070E00026C78ECFF89410926F0010928100109285001092840081E085BF15BE47985D9AEB
:20710000289A0C94000008952091B2013091B3012F5F3F4F3093B3012093B201932F37FFA6
:2071200003C08EEF831B982F990F921710F447980895479A08951F920F920FB60F9211246E
:207140002F938F939F93EF93FF9310928500109284008091A8019091A901009741F00197D3
:207160009093A9018093A801892B09F45D9A8091AA019091AB01009741F001979093AB0126
:207180008093AA01892B09F4289AE0E0F0E0859194918F5F9F4F49F08091AC019091AD0151
:2071A00001969093AD018093AC01FF91EF919F918F912F910F900FBE0F901F90189584E0BC
:2071C0008093E9000DC08091E8008B778093E80003C08EB3882351F08091E80082FFF9CFBE
:2071E0008091E80085FFEFCF8091F1000895982F83E08093E9008091E80085FD0DC0809136
:20720000E8008E778093E80003C08EB3882369F08091E80080FFF9CF9093F1005D9884E6CB
:2072200090E09093A9018093A80108954F925F926F927F928F929F92AF92BF92CF92DF921E
:20724000EF92FF920F931F93CF93DF9384E08093E9008091E80082FF57C2289884E690E067
:207260009093AB018093AA01AADF182F853481F48CE49DE19093AD018093AC0107B600FC4B
:20728000FDCFF999FECF81E180935700E89503C0843519F494DF8DE00DC28C34E1F38035F9
:2072A000D1F3843721F484E4A2DF80E003C2813611F489E5FFC18134B1F481DF182F7FDFE3
:2072C00090E0880F991FAA2797FDA095BA2F312F330F20E0442737FD4095542F822B932B68
:2072E000A42BB52BB8C1803711F483E5E3C1833549F4C0E0D1E089917ADF21E0C730D20714
:20730000D1F7D9C1863521F481E371DF80E3D2C1833731F487E86BDF85E969DF8EE1CAC149
:207320008536B9F4E0E0F0E093E085E090935700E89507B600FCFDCF80935700E89507B65D
:2073400000FCFDCFE058FF4FA0E7E030FA0771F7A2CF823739F4E1E0F0E089E08093570024
:207360008491A8C1863439F4E0E0F0E089E08093570084919FC18E3439F4E3E0F0E089E0E5
:2073800080935700849196C1813539F4E2E0F0E089E08093570084918DC1823631F489E521
:2073A00026DF80E024DF80E885C1823419F0873609F0E5C01092AD011092AC0100DF082FE8
:2073C000FEDEF82EFCDE682E8554823008F071C1902F80E0CF2DD0E0C82BD92B10926F00B3
:2073E000173609F04BC081E180935700E895DD24CC24C3943FC0E090AE01F090AF010091CC
:20740000B0011091B101B6E46B16D9F4ED2DF0E0EE29FF29E4918E2FEADEDD2081F082E08D
:2074200090E0A0E0B0E0E80EF91E0A1F1B1FE092AE01F092AF010093B0011093B101DC2470
:2074400018C0D801C701B695A7959795879559D5CEDE82E090E0A0E0B0E0E80EF91E0A1FF2
:207460001B1FE092AE01F092AF010093B0011093B1012197209709F0BECF7DC08090AE01F5
:207480009090AF01A090B001B090B10196E4691609F05DC083E0F40180935700E89507B63E
:2074A00000FCFDCF54C0F6E46F1661F5772031F1E090AE01F090AF010091B0011091B1019E
:2074C0007EDED82ECC24852D90E08C299D29F7010C0140925700E895112482E090E0A0E08B
:2074E000B0E0E80EF91E0A1F1B1FE092AE01F092AF010093B0011093B10102C060DE582E1A
:20750000742423C0E090AE01F090AF010091B0011091B10116950795F794E79450DE682FFA
:20752000C701F7D48091AE019091AF01A091B001B091B1010296A11DB11D8093AE01909349
:20754000AF01A093B001B093B101219704C05524772444244394209709F0A5CF96E46916B6
:2075600041F485E0F40180935700E89507B600FCFDCF8DE03CDE82E080936F009CC0833492
:2075800071F40091AE011091AF0119DE90E021E0F8010C0120935700E89511247CCE8336C8
:2075A00019F5E090AE01F090AF010091B0011091B10105DEF701E16090E021E00C0120938C
:2075C0005700E895112482E090E0A0E0B0E0E80EF91E0A1F1B1FE092AE01F092AF0100936A
:2075E000B0011093B10157CE8D3661F4E091AE01F091AF0185E080935700E89507B600FCF2
:20760000FDCF49CE823551F4E091AE01F091AF0105911491812FEBDD802F4CC0843421F5FE
:20762000E090AE01F090AF010091B0011091B10116950795F794E794C2DD682FC70169D4DE
:207640008091AE019091AF01A091B001B091B1010296A11DB11D8093AE019093AF01A093D8
:20766000B001B093B10117CE843609F5E090AE01F090AF010091B0011091B101D801C70142
:20768000B695A795979587953CD4B1DD82E090E0A0E0B0E0E80EF91E0A1F1B1FE092AE010A
:2076A000F092AF010093B0011093B10104C08B3111F08FE39CDD83E08093E9009091E8002B
:2076C0008091E8008E778093E80095FF04C010C08EB38823C9F08091E80080FFF9CF809193
:2076E000E8008E778093E80003C08EB3882361F08091E80080FFF9CF84E08093E9008091F1
:20770000E8008B778093E800DF91CF911F910F91FF90EF90DF90CF90BF90AF909F908F90AC
:207720007F906F905F904F9008959091B601892F8F77813249F58091B7018032A1F081328A
:2077400019F5913A09F58091E800877F8093E8008DE091E067E070E00BD28091E8008B770B
:207760008093E8000895913279F48091E800877F8093E8008DE091E067E070E05DD2809192
:20778000E8008E778093E800089582E061EC42E0B5D083E061E842E1B1D084E060E842E1EF
:2077A000ADC084B7877F84BF88E10FB6F89480936000109260000FBE20E880E090E00FB63F
:2077C000F89420936100809361000FBE81E085BF92E095BF3F9A209A559AE1E6F0E02083A1
:2077E000108247985D9A289A109289008AEF8093880090936F0083E080938100F0C0409116
:20780000000850910108109201081092000894B714BE88E10FB6F8948093600010926000D5
:207820000FBE292F30E0F901E270F07091FD18C090FF05C0859194918F5F9F4F81F423FFFF
:207840000FC08091090190910A014817590741F0E0E0F0E0859194918F5F9F4F09F042DC64
:20786000A0DF78941092AD011092AC010CC0DEDC36D38091AC019091AD0181549F4110F00D
:207880001092140141DC80911401882381F78091E00081608093E00025DC80E090E0089598
:2078A000FA01923049F0933061F09130F9F485E191E022E130E01EC087E291E02EE330E04D
:2078C00019C0882329F485E691E024E030E012C0813029F489E691E022E230E00BC0823006
:2078E00029F48DE891E028E130E004C080E090E020E030E091838083C90108958093E9004E
:207900008091EB0081608093EB001092ED006093EC004093ED008091EE00881F8827881F62
:2079200008958091B60188238CF403C08EB38823B1F08091E80082FFF9CF8091E8008B772A
:207940008093E80008958EB3882349F08091E80080FFF9CF8091E8008E778093E800089594
:20796000EF92FF920F931F9345D04CD008ED10E0F80180818F77808380818068808380819B
:207980008F7D808319BC1EBA1092B40180EEE82EF12CF70180818B7F8083F8018081816052
:2079A000808380E060E042E0A9DFE1EEF0E080818E7F8083E2EEF0E0808181608083808144
:2079C00088608083F70180818E7F8083F8018081806180831F910F91FF90EF900895E7ED06
:2079E000F0E08081816080838AE482BF81E08093B501B6CFE8EDF0E080818E7F808310921C
:207A0000E20008951092DA001092E10008951F920F920FB60F9211242F933F934F935F93F6
:207A20006F937F938F939F93AF93BF93EF93FF938091DA0080FF1BC08091D80080FF17C0B2
:207A40008091DA008E7F8093DA008091D90080FF0BC080E189BD82E189BD09B400FEFDCF36
:207A600081E08EBB3BD203C019BC1EBA37D28091E10080FF17C08091E20080FF13C0809138
:207A8000E2008E7F8093E2008091E20080618093E2008091D80080628093D80019BC85E049
:207AA0008EBB1CD28091E10084FF2CC08091E20084FF28C080E189BD82E189BD09B400FEC5
:207AC000FDCF8091D8008F7D8093D8008091E1008F7E8093E1008091E2008F7E8093E20012
:207AE0008091E20081608093E2008091B401882331F48091E30087FD02C081E001C084E067
:207B00008EBBECD18091E10083FF21C08091E20083FF1DC08091E100877F8093E10082E06A
:207B20008EBB1092B4018091E1008E7F8093E1008091E2008E7F8093E2008091E2008061E9
:207B40008093E20080E060E042E0D8DEC7D1FF91EF91BF91AF919F918F917F916F915F9130
:207B60004F913F912F910F900FBE0F901F9018959C014091BC015091BD014617570718F49D
:207B8000F90190E044C06115710511F0AB01F8CF8091E8008E778093E80040E050E0F0CF0F
:207BA0008EB3882309F444C0853009F443C08091E80083FF02C081E008958091E80082FD70
:207BC00031C08091E80080FF22C08091F3009091F200782F60E0292F30E0262B372B07C07A
:207BE00081918093F100415050402F5F3F4F4115510519F02830310598F390E02830310566
:207C000009F491E08091E8008E778093E8004115510531F6992321F605C08EB3882341F075
:207C2000853041F08091E80082FFF7CF80E0089582E0089583E008959C016115710529F47C
:207C40008091E8008B778093E800F90126C08EB3882391F1853091F18091E80083FF02C06C
:207C600081E008958091E80082FFF1CF06C08091F10081936150704059F02091F300809191
:207C8000F200322F20E090E0822B932B892B79F78091E8008B778093E80061157105B9F601
:207CA00005C08EB3882341F0853041F08091E80080FFF7CF80E0089582E0089583E00895C2
:207CC0000F931F93DF93CF9300D0CDB7DEB7E6EBF1E08091F100819381E0EE3BF807C9F792
:207CE00024DD8091E80083FFE4C08091B6019091B701953009F46DC0963040F4913081F1A7
:207D0000913070F0933009F0D4C02AC0983009F4A3C0993009F4B2C0963009F0CAC07CC023
:207D2000803809F4C6C0823809F0C3C08091BA0187708093E9008091EB001092E9002091DB
:207D4000E800277F2093E80090E025E0969587952A95E1F781708093F1001092F10087C0D8
:207D6000882319F0823009F0A4C08F71823009F0A0C08091B801882331F52091BA01277097
:207D800009F497C02093E9008091EB0080FF1BC0933021F48091EB00806213C08091EB0018
:207DA00080618093EB0081E090E002C0880F991F2A95E2F78093EA001092EA008091EB00E5
:207DC00088608093EB001092E9008091E800877F51C0882309F06DC01091B8011F770FB79B
:207DE000F8948091E800877F8093E8009ADD8091E80080FFFCCF8091E3008078812B809398
:207E0000E30080688093E300112311F482E001C083E08EBB0FBF4DC08058823008F049C033
:207E20008091B8019091B9016091BA01AE014F5F5F4F36DDBC01009709F43BC08091E8008E
:207E4000877F8093E80089819A8192DE8091E8008B778093E8002DC0803859F58091E800AA
:207E6000877F8093E8008091B4018093F1008091E8008E778093E80054DD1BC08823C9F4CA
:207E80009091B8019230A8F48091E800877F8093E8009093B40145DD8091B401882331F420
:207EA0008091E30087FD02C081E001C084E08EBB6CDC8091E80083FF0AC08091EB0080624E
:207EC0008093EB008091E800877F8093E8000F900F90CF91DF911F910F91089508951F9360
:207EE0008EB3882361F01091E9001092E9008091E80083FF01C0E4DE17701093E9001F916F
:207F00000895F999FECF92BD81BDF89A992780B50895262FF999FECF1FBA92BD81BD20BDBD
:207F20000FB6F894FA9AF99A0FBE01960895F894FFCF4341544552494E4100777700080031
:207F40000000000000080112011001020000084123360001000201000109023E00020100FF
:207F600080320904000001020201000524001001042402040524060001070582030800FF0C
:207F800009040100020A000000070504021000010705830210000104030904220341007216
:207FA000006400750069006E006F0020004C0065006F006E006100720064006F0000001836
:1A7FC00003410072006400750069006E006F0020004C004C004300000000D7
:00000001FF
